:100000000C9426050C9441050C9441050C94410573
:100010000C9441050C9441050C9441050C94410548
:100020000C9441050C94350D0C9441050C9441053C
:100030000C9441050C9441050C9441050C94410528
:100040000C9441050C9441050C9441050C94410518
:100050000C9441050852573F9F5A49CBA5620F7631
:10006000C76913F27E6F500D0175360B617A2AAAAB
:10007000AB7E0000007F00000000696E69743A00EA
:100080004E5450203A203C72657175657374206F30
:1000900075743E0D0A00554450203A203F0D0A0069
:1000A0000D0A00415250203A20616464696E672055
:1000B0006970200020746F206D6163207461626C30
:1000C0006500415250203A2077686F2068617320A4
:1000D000002074656C6C2000415250203A20676FFC
:1000E00074207265706C7920666F722075730041A0
:1000F0005250205441424C453A00202020207C2080
:100100004D4143202020202020202020202020207E
:10011000202020202020207C20495000207C20000E
:10012000207C20007074723A20004E4943203A200F
:10013000656E6332386A363020696E69742E2E2EF1
:100140002000646F6E650D0A004E4943203A20007E
:100150001F1D1F1E1F1E1F1F1E1F1E1F4E5450201F
:100160003A206E7470207365727665722000206F7D
:1001700075747369646520686F6D65206E657420A1
:100180002D3E2075736520676174657761790D0A6E
:10019000004E5450203A2074696D657374616D701F
:1001A0002069732000444154453A20002054494DB1
:1001B000453A2000202855544321290049434D50F9
:1001C0003A206563686F207265706C792073656E84
:1001D0007400434C4B203A20696E697420646F6E42
:1001E000652E0D0A00434C4B203A20000D0A0000FA
:1001F0005EBCE2613FDD83C29C7E20A3FD1F419D6A
:10020000C3217FFCA2401E5F01E3BD3E6082DC2370
:100210007D9FC1421CFEA0E1BF5D0380DE3C62BE4B
:10022000E0025CDF81633D7C22C09E1D43A1FF464E
:1002300018FAA427799BC584DA3866E5BB5907DB31
:10024000856739BAE406581947A5FB7826C49A652C
:100250003BD987045AB8E6A7F91B45C6987A24F813
:10026000A6441A99C7257B3A6486D85B05E7B98C02
:10027000D2306EEDB3510F4E10F2AC2F7193CD1101
:100280004FADF3702ECC92D38D6F31B2EC0E50AFD8
:10029000F1134DCE90722C6D33D18F0C52B0EE32E3
:1002A0006C8ED0530DEFB1F0AE4C1291CF2D73CABE
:1002B000947628ABF517490856B4EA6937D58B57B9
:1002C00009EBB536688AD495CB2977F4AA4816E9A4
:1002D000B7550B88D6346A2B7597C94A14F6A8749B
:1002E0002AC896154BA9F7B6E80A54D7896B356327
:1002F000206279206176722E61756374696F6E6118
:100300006E742E64650400050006000706080209E5
:10031000060AFF0B1FC100C00DC232CAEECB05C4D6
:1003200012C612C70CE4ACE5DEE248E3AAE0BBE18A
:10033000CC544350203A2054544C2074696D656F5E
:10034000757420666F7220736F636B6574205B0039
:100350005D2E20736F636B657420636C6F736564CF
:100360002E00544350203A2069702000206F75748D
:100370007369646520686F6D65206E6574202D3E1D
:100380002075736520676174657761790D0A005483
:100390004350203A204552522041525020554B4E56
:1003A000574E3A20002D3E2063616C6C696E6720C9
:1003B000617270276861636B20746F2061646420D0
:1003C0006D61633C2D3E6970206D617070696E6770
:1003D00000544350203A2069676E6F72696E67203F
:1003E0007061636B657420666F72206970200054C1
:1003F0004350203A20736F636B65745B005D202D62
:100400003E20002052535420464C414720726563E1
:100410006569766564202D3E20736F636B6574207B
:10042000434C4F5345442E0D0A0045535441424C12
:10043000495348454400434C4F534544004C4153B5
:10044000545F41434B00544350203A2061636B207A
:10045000213D206C617374207365716E756D212070
:1004600072657472616E736D6974203A2000205752
:1004700041524E3A20746370206461746120647547
:1004800070212069676E6F72696E67206475706C89
:10049000696361746520646174612E200020455297
:1004A00052203A20746370207061636B6574206C15
:1004B0006F7374212072652D72657175657374692F
:1004C0006E672E200044415441205452414E534601
:1004D0004552200020627974657300445B004C41F2
:1004E00053545F41434B004C4153545F41434B2DA8
:1004F0003E434C4F5345440046494E5F5741495493
:10050000312D3E00434C4F53494E470054494D4511
:10051000445F574149540046494E5F574149543260
:100520000046494E5F57414954322D3E54494D458E
:10053000445F574149540054494D45445F57414930
:10054000543A207061636B657420696E203F2120EE
:1005500000434C4F53494E472D3E54494D45445F4F
:1005600057414954004552524F523A20696E7661C4
:100570006C69642074637020737461746520212039
:10058000736F636B657420636C6F736564210054D3
:10059000494D45445F574149543A2074696D656F30
:1005A00075742073657420746F2035732000544374
:1005B00050203A20636F6E6E656374696F6E2072AF
:1005C0006571756573742E205B4F4B5D005443500D
:1005D000203A205741524E3A2069676E6F72696E19
:1005E00067207061636B657420286E6F20736F6382
:1005F0006B6574206F70656E29003C68746D6C3E8D
:100600003C626F64793E3430343A2066696C652010
:100610006E6F7420666F756E643C68723E617672B0
:1006200045544831207765627365727665723C2F58
:10063000626F64793E3C2F68746D6C3E003C687458
:100640006D6C3E3C626F64793E3C62723E3C636519
:100650006E7465723E3C646976207374796C653D96
:1006600027666F6E742D73697A653A203230307068
:10067000743B20636F6C6F723A20234646464646B1
:10068000463B206261636B67726F756E643A20232C
:10069000303030303030273E68656C6C6F3C2F64F2
:1006A00069763E3C646976207374796C653D276693
:1006B0006F6E742D73697A653A2032303070743BF6
:1006C000273E776F726C643C2F6469763E3C6272A1
:1006D0003E3C696D67207372633D222F67726170C3
:1006E000683022206865696768743D22313336229C
:1006F0002077696474683D22353736223E3C2F638B
:10070000656E7465723E3C2F626F64793E3C2F6863
:10071000746D6C3E000D0A0D0A00696D6167652FEE
:10072000626D7000746578742F68746D6C00485445
:1007300054502F312E3020343034206E6F742066A8
:100740006F756E640D0A5365727665723A20617634
:1007500072455448310D0A436F6E74656E742D54A2
:100760007970653A20746578742F68746D6C0048F0
:100770005454502F312E302032303020446F637566
:100780006D656E7420666F6C6C6F77730D0A5365C0
:10079000727665723A20617672455448310D0A438B
:1007A0006F6E74656E742D547970653A20004854EC
:1007B00054503A2072657175657374656420646184
:1007C00074612062797465205B002D3F5D0D0A0025
:1007D0000D0A474554203C003E2E0D0A00696E6408
:1007E000657800677261706830003C68746D6C3EBB
:1007F0003C626F64793E75706C6F6164205B2E00A3
:10080000696E6465782E2E2E0067656E20626D70AD
:100810002E2E2E0034303421000000000000000095
:1008200000000000000000000000000000000000C8
:100830000000000000000000000000000003C38072
:10084000020440E104470084400044400246400165
:100850008380000000000000000000000000000095
:100860000000000000000000000001C38000844080
:1008700070844700844000844001864000838000EB
:100880000000000000000000000000000000000068
:100890000000000000000000038000044000044746
:1008A00000044000044000064000038000000000F7
:1008B0000000000000000000000000000000000038
:1008C0000000000001C38000844000844700844091
:1008D000008440018640008380000000000000008A
:1008E0000000000000000000000000000000000008
:1008F0000003C380020440010447008440004440D8
:10090000024640018380000000000000000000005B
:100910000000000000000000000000000000038351
:100920008002444000444700C440018440004640E7
:1009300003838000000000000000000000000000B1
:1009400000000000000000000000000043800044A0
:100950004003E44701444001444000C64000438056
:100960000000000000000000000000000000000087
:10097000000000000000000003C380026440002467
:100980004702244003C44002064003C38000000025
:10099000000000000000000000000000001C00003B
:1009A0002000002000021000050C00020000424D53
:1009B0007E260000000000003E000000280000002D
:1009C000400200008800000001000100000000005B
:1009D00040260000110B0000110B00000200000077
:1009E00002000000FFFFFF00FF000000793A200036
:1009F000783A20006874747020636C69656E740DB9
:100A00000A00474554202F73747265616D2F313091
:100A1000343020485454502F312E310D0A486F7312
:100A2000743A2036342E3233362E33342E31393662
:100A30003A38300D0A4163636570743A2074657802
:100A4000742F68746D6C0D0A0D0A000011241FBE0E
:100A5000CFE5D8E0DEBFCDBF10E0A0E6B0E0E0ED2E
:100A6000FCE302C005900D92A037B107D9F714E05E
:100A7000A0E7B0E001C01D92AE30B107E1F70C94E1
:100A800043050C940000CFE5D8E0DEBFCDBF8FEF6B
:100A900087BB84BB88BBA89A40E050E0E12C68E4A7
:100AA000F62E012D112DAB9A27E030E0C7010197FA
:100AB000F1F72150304037FFF9CFAB98A0E0B8E410
:100AC000C0E0D0E027E030E0CD010197F1F7215000
:100AD000304037FFF9CF4F5F5F4F4530510518F376
:100AE0000E94AE060E94500E8AE790E00E942A0EF5
:100AF0000E94D7090E94DB0A0E94240D0E948211E5
:100B0000A0E0B4E2C0E0D0E023E630E0CD01019700
:100B1000F1F72150304037FFF9CF80E790E00E9495
:100B2000EA0A80E890E00E942A0E0E94E2180E94E1
:100B30008C1B68E572E080E790E00E94130ABC011C
:100B4000181619060CF057C080917C009927382F91
:100B5000222780917D00280F311D88E0263038073C
:100B600071F480E790E00E940908809104038130CD
:100B700009F041C080E790E00E94EA0A3CC02050A2
:100B80003840C9F5C09187008C2F99278630910590
:100B900071F0873091051CF4019721F023C0419733
:100BA00059F020C080E790E00E94B60C24C080E796
:100BB00090E00E94E0121FC0809194009927982F26
:100BC000882720919500820F911D8B5B9C4929F409
:100BD00080E790E00E94110C0EC086E990E00E9430
:100BE0002A0E09C080E690E00E94410E8C2F0E94E0
:100BF000AD0D0E943C0E80910903813009F099CF20
:100C00000E94AE111092090394CF5D9BFECF8CB968
:100C100080E090E008950F931F93CF93182F00E08A
:100C2000C4E680E390E01C1730F001E01C1B019645
:100C30001C17E0F708C0002331F48033910519F444
:100C4000C13009F080E20E9405068C2F6AE00E9404
:100C5000261EC82F882329F7CF911F910F91089541
:100C6000EF92FF920F931F937B018C01892F99279D
:100C7000AA27BB270E940B068EE20E940506C80128
:100C8000AA27BB270E940B068EE20E940506BB27FF
:100C9000A12F902F8F2D0E940B068EE20E94050639
:100CA0008E2D0E940B061F910F91FF90EF900895DB
:100CB000FF920F931F93CF93DF938C01FF24C0E12A
:100CC000D7E280E390E00C171D0748F031E0F32EE7
:100CD0000C1B1D0B01960C171D07D0F709C0FF2038
:100CE00039F48033910521F4C130D10509F080E257
:100CF0000E940506CE016AE070E00E94321EEB0100
:100D0000672BF9F6DF91CF911F910F91FF90089516
:100D1000CF93DF93EC01FC0121968491882339F075
:100D20000E940506FE01219684918823C9F7DF9170
:100D3000CF91089580EA90E00E9488060895CF93AD
:100D4000DF93EC018881882331F089910E940506A8
:100D500088818823D1F7DF91CF910895539A80B588
:100D6000866880BD10BC83E089B90895CF92DF9278
:100D7000EF92CF93DF93EC01CA0196012C5E3F4FB7
:100D80005AEFC52E52E0D52EAC01FE01DA018D914D
:100D9000AD018083D6018D916D0186833196BFEFC1
:100DA000CB16B2E0DB0691F388F388E08C871D86D2
:100DB00085E48E871F86832F9927888B298B8091C6
:100DC000CA029091CB02892F99278A8B8091CA02FF
:100DD0009091CB028B8B8091CA029091CB020196AD
:100DE0009093CB028093CA0280E48C8B1D8A80E8AA
:100DF0008E8BEF8AFB014081518162817381CE012C
:100E00004E960E944B0A8091000390910103A0919D
:100E10000203B0910303AC01BD01CE014A960E94CA
:100E20004B0A188E198E20E030E040E050E064E17B
:100E300070E0CE010E960E949C0A9C01832F992798
:100E4000888F298FDF91CF91EF90DF90CF90089519
:100E50004F925F926F927F928F929F92AF92BF92CA
:100E6000CF92DF92EF92FF920F931F935C013901B3
:100E70002801470128E030E0820E931E640131E131
:100E8000E32E9301C5010E94B606872D9927F5012F
:100E900082A363A2852D992784A345A2892D992732
:100EA00086A387A210A611A61F910F91FF90EF9025
:100EB000DF90CF90BF90AF909F908F907F906F907A
:100EC0005F904F90089580E090E09C0143E0FC012A
:100ED000E20FF31FE253FD4F108211821282138240
:100EE00041502F5F3F4F099647FFF1CF1092CD023F
:100EF0001092CC020895EF92FF920F931F937B0103
:100F00008C0120E030E0A901FA01E20FF31FE25367
:100F1000FD4F80819181A281B3818E159F05A0072D
:100F2000B10711F4C90109C02F5F3F4F475F5F4F01
:100F3000243031054CF38FEF9FEF1F910F91FF90FD
:100F4000EF900895CF92DF92EF92FF920F931F934D
:100F50006C017A018B0183EA90E00E942A0EC8019D
:100F6000B7010E94D20D84EB90E00E942A0E0E94ED
:100F70003C0E8091CC029091CD02FC0163E0EE0F1B
:100F8000FF1F6A95E1F7E80FF91FE80FF91FE25319
:100F9000FD4FE082F18202831383D60120E030E02E
:100FA00045E08091CC029091CD02FC0153E0EE0F20
:100FB000FF1F5A95E1F7E80FF91FE80FF91FE253F9
:100FC000FD4FE20FF31F8D91848341502F5F3F4F00
:100FD00047FFE7CF2091CC023091CD028091CC0227
:100FE0009091CD0201969093CD028093CC02809196
:100FF000CC029091CD02049724F01092CD02109271
:10100000CC02C9011F910F91FF90EF90DF90CF901C
:1010100008954F925F926F927F928F929F92AF92BC
:10102000BF92CF92DF92EF92FF920F931F93CF93D5
:10103000DF93EC012B01FCE18F2E912C880E991E81
:10104000C4010E94200A5B016C01E6E26E2E712C45
:101050006C0E7D1EC3010E94200A7B018C01CE0113
:101060000E94160A019709F08FC0809100039091A9
:101070000103A0910203B0910303E816F9060A07E1
:101080001B0709F0B5C082EC90E00E942A0EC8014F
:10109000B7010E94D20D81ED90E00E942A0EC60198
:1010A000B5010E94D20D0E943C0EC601B5010E94FE
:1010B0007B079C0197FF17C02091CC023091CD0295
:1010C0008091CC029091CD0201969093CD028093B5
:1010D000CC028091CC029091CD02049724F0109222
:1010E000CD021092CC02C90173E0880F991F7A9546
:1010F000E1F7FC01E20FF31FE20FF31FE253FD4F94
:10110000A082B182C282D382F901E20FF31FE80FFD
:10111000F91FEE52FD4FDE01569695E08D918193B9
:10112000915097FFFBCFCE0106960E94C909FE01A0
:1011300095E086898193915097FFFBCF1C8A82E0CE
:101140008D8BFE0195E0868980A39150319697FFA3
:10115000FACFCE0146960E94C90980910003909172
:101160000103A0910203B0910303AC01BD01C401CE
:101170000E944B0AB601A501C3010E944B0AB201AD
:10118000CE010E94100A34C0CE010E94160A0297B6
:1011900079F5C3010E94200A9B01AC0180910003F4
:1011A00090910103A0910203B0910303281739071E
:1011B0004A075B07E9F488ED90E00E942A0E0E943E
:1011C0003C0EC401AA2797FDA095BA2FBC01CD0102
:1011D0000E947B078F5F9F4F59F4C4010E94200A31
:1011E000DC01CB01AC01BD01CE0146960E94A207F5
:1011F000DF91CF911F910F91FF90EF90DF90CF90F3
:10120000BF90AF909F908F907F906F905F904F9026
:101210000895FF920F931F93CF93DF93EC018B01FF
:10122000AFEFFA2EAAEFB2E0FC0125E0F0828D913B
:1012300086832150319627FFF9CF26E088E08C87FE
:101240002D871E8691E09F87888B198A2A8B84E0E0
:101250008B8B1C8A9D8BCE0146960E94C90980917A
:10126000000390910103A0910203B0910303AC012C
:10127000BD01CE014C960E944B0A8F2DFE01B09607
:1012800025E08193215027FFFCCFF8014081518157
:1012900062817381CE0186960E944B0A6AE270E0F9
:1012A000CE010E94100ADF91CF911F910F91FF9004
:1012B0000895AF92BF92CF92DF92EF92FF920F9379
:1012C0001F93CF93DF938FEE90E00E942A0E0E942F
:1012D0003C0E8AEF90E00E942A0E0E943C0EEE2403
:1012E000FF24570167018E2D0E94AD0D8CE191E026
:1012F0000E942A0EF601EE0DFF1DE253FD4F848180
:101300000E94AD0D01E010E08AE30E94910DE5011D
:10131000CE0DDF1DC253DD4FFE01E00FF11F8481B2
:101320000E94AD0D0F5F1F4F063011056CF380E278
:1013300091E00E942A0E688179818A819B810E94B6
:10134000D20D0E943C0E0894E11CF11C89E090E053
:10135000C80ED91EA80EB91E94E0E916F1041CF2BD
:1013600084E291E00E942A0E8091CC029091CD02FD
:101370000E94AD0D0E943C0E0E943C0EDF91CF9169
:101380001F910F91FF90EF90DF90CF90BF90AF90A3
:101390000895FC018CEA80838EED818388E482834A
:1013A0008AEA83838BEB84838CEC858308958AE2BD
:1013B00091E00E942A0E0E94151182E491E00E94A1
:1013C0002A0E8AEF92E00E94C90986E090E0A8EA1E
:1013D000B0EC8093000390930103A0930203B093B9
:1013E000030389E491E00E942A0E8091000390910A
:1013F0000103A0910203B0910303BC01CD010E943F
:10140000D20D0E943C0E82E490E0A8EAB0EC8093FA
:10141000F6029093F702A093F802B093F9020895B0
:101420000E94241008950E949B100895FC01848955
:101430009927382F222785899927822B932B089566
:10144000FC0180819927AA27BB27B82FAA279927B3
:1014500088272181332744275527A90133272227AD
:10146000822B932BA42BB52B22813327442755277E
:10147000542F432F322F2227822B932BA42BB52BB3
:101480002381332744275527822B932BA42BB52B5D
:10149000BC01CD010895FC019A01AB01852F99276C
:1014A000AA27BB278083CA01AA27BB278183BB2722
:1014B000A52F942F832F828323830895FC0180819D
:1014C0009927AA27BB27B82FAA27992788272181E0
:1014D000332744275527A90133272227822B932B13
:1014E000A42BB52B2281332744275527542F432F74
:1014F000322F2227822B932BA42BB52B238133272A
:1015000044275527822B932BA42BB52BBC01CD014F
:101510000895FC019A01AB01852F9927AA27BB27C3
:101520008083CA01AA27BB278183BB27A52F942FBD
:10153000832F828323830895CF93DF93EC01FB01F4
:10154000BA01A901E230F10578F089912991992732
:10155000982F8827820F911DAA27BB27480F591F54
:101560006A1F7B1F3297EECFEF2B51F088819927AE
:10157000982F8827AA27BB27480F591F6A1F7B1F50
:10158000DB01CA01A070B070AB0166277727480F56
:10159000591F6A1F7B1FDB01CA01A070B0709B013D
:1015A00044275527820F931FA41FB51F8095909540
:1015B000DF91CF91089581E49CE1AEE8B0E480939F
:1015C000050390930603A0930703B09308031092BA
:1015D00004030895EF92FF920F931F93CF93DF932D
:1015E000EC0183EE8AA71BA684E08CA78AEF8DA767
:1015F000FE01BE96CE01875A9F4F11928E179F070C
:10160000E0F781E08FA78BAB2091050330910603B3
:10161000409107035091080320708091000390913E
:101620000103A0910203B0910303807028173907CA
:101630004A075B07B9F08CE591E00E942A0E809181
:10164000050390910603A0910703B0910803BC0124
:10165000CD010E94D20D8EE691E00E942A0E06EF87
:1016600012E002C005E013E0F8016081718182811F
:1016700093810E947B079C01FFEF8F3F9F0741F4FE
:10168000B801CE010E94090981E0809304031FC0C4
:101690001092040343E0880F991F4A95E1F7820FE7
:1016A000931F820F931F8E529D4F20E3E22EF12C49
:1016B0000BE710E02BEB3CE9AC0165E073E0CE01F9
:1016C0000E9428076AE570E0CE010E94100ADF91AF
:1016D000CF911F910F91FF90EF900895EF92FF929D
:1016E0000F931F93CF93DF937B018C01EA012CE3CF
:1016F00030E040E050E00E94461EDC01CB018D83CB
:10170000C801B7012CE330E040E050E00E94461EE3
:1017100079018A01CA01B9012CE330E040E050E0D0
:101720000E94461EDC01CB018C83C801B7012CE36B
:1017300030E040E050E00E94461E79018A01CA0173
:10174000B90128E130E040E050E00E94461EDC0193
:10175000CB018B83C801B70128E130E040E050E0C5
:101760000E94461E79018A01C801AA27BB270E9450
:101770005806C7010E94580640E054E02DE631E0CB
:10178000842F992783709070892B61F42EE631E0C5
:10179000442321F0443611F0483C21F4515011F01B
:1017A0002DE631E0C901AA27BB27E816F9060A078A
:1017B0001B0730F0E81AF90A0A0B1B0B4F5FDECF4C
:1017C00048832D56314059F4EBE3EE16F104010540
:1017D000110528F00894E11CF11C011D111D20E5E4
:1017E00031E041E0F9012F5F3F4F8491E81AF108A1
:1017F00001091109F90184919927AA27BB27E81645
:10180000F9060A071B0718F04F5F4C3058F3EA82BD
:101810004F5F4983DF91CF911F910F91FF90EF9020
:101820000895AF92BF92CF92DF92EF92FF920F9303
:101830001F93CF93DF93CDB7DEB726970FB6F894FB
:10184000DEBF0FBECDBFFC0182A599278F739070BC
:10185000849709F07AC08F010E5A1F4FD8018C91DE
:101860009927982F8827AA2797FDA095BA2FED5A78
:10187000FF4F2191820F911DA11DB11DBA2FA92FDC
:10188000982F88272191820F911DA11DB11DCC2475
:10189000D82EE92EFA2E8081C80ED11CE11CF11C35
:1018A00081E991E00E942A0E580103E010E0F50161
:1018B00081915F010E94AD0D80E20E94910D015067
:1018C000104017FFF4CF0E943C0EAE014F5F5F4FF8
:1018D000C701B6010E946E0B85EA91E00E942A0EB4
:1018E0008B810E94AD0D8EE20E9405068A810E94C6
:1018F000AD0D8EE20E940506898199278459984F83
:101900000E94FA0D8CEA91E00E942A0E8C810E94BE
:10191000AD0D8AE30E9405068D810E94AD0D8AE31C
:101920000E9405068E810E94AD0D84EB91E00E941D
:101930002A0E8C818F5F80930A038D8180930B0325
:101940008E8180930C030E943C0E26960FB6F8946D
:10195000DEBF0FBECDBFDF91CF911F910F91FF90E2
:10196000EF90DF90CF90BF90AF900895EF92FF92ED
:101970000F931F93CF93DF93EC017B018AA18830F3
:1019800009F05BC08CEB91E00E942A0E0E943C0E95
:101990008E01065E1F4FC8010E94200ADC01CB01A8
:1019A000BC01CD010E947B0797FF0AC0FE019E018A
:1019B0002B5F3F4F868181932E173F07DCF715C0C1
:1019C000DE01FC0123E0EE0FFF1F2A95E1F7E80F8F
:1019D000F91FE80FF91FEE52FD4F9E012B5F3F4F9D
:1019E00081918D932A173B07DCF7CE0106960E9462
:1019F000C9091AA29CA1983F18F08DA18F5F8DA3F1
:101A0000985F9CA3FE019E012D5F3F4F828D868FC4
:101A100031962E173F07D4F7809100039091010370
:101A2000A0910203B0910303AC01BD01C8010E9463
:101A30004B0AB701CE010E94100ADF91CF911F918E
:101A40000F91FF90EF9008951092090384E089BFF1
:101A50008EB585608EBD8FED93EE9DBD8CBD789467
:101A600082ED91E00E942A0E08951F920F920FB608
:101A70000F9211242F933F934F935F936F937F9314
:101A80008F939F93AF93BF93EF93FF938FED93EE5D
:101A90009DBD8CBD81E08093090380910C038F5F15
:101AA00080930C038C33A1F410920C0380910B03F0
:101AB0008F5F80930B038C3359F410920B0380914A
:101AC0000A038F5F80930A03883111F410920A038E
:101AD00085EE91E00E942A0E80910A030E94AD0DCE
:101AE0008AE30E94910D80910B030E94AD0D8AE361
:101AF0000E94910D80910C030E94AD0D0E943C0E3E
:101B0000FF91EF91BF91AF919F918F917F916F91D5
:101B10005F914F913F912F910F900FBE0F901F90AB
:101B20001895682F78E0A8988FE790E0A0E0B0E0E3
:101B3000282F2A95F1F79C01AD0160FF02C0A89AF9
:101B400001C0A898822F8A95F1F766957150A9F780
:101B5000A89A8FE78A95F1F708950F931F93CF9373
:101B6000182F00E0C4E680E390E01C1730F001E09D
:101B70001C1B01961C17E0F708C0002331F48033CA
:101B8000910519F4C13009F080E20E94910D8C2F6B
:101B90006AE00E94261EC82F882329F7CF911F9143
:101BA0000F910895EF92FF920F931F937B018C0189
:101BB000892F9927AA27BB270E94AD0D8EE20E948C
:101BC000910DC801AA27BB270E94AD0D8EE20E948D
:101BD000910DBB27A12F902F8F2D0E94AD0D8EE26E
:101BE0000E94910D8E2D0E94AD0D1F910F91FF90BF
:101BF000EF900895FF920F931F93CF93DF938C0183
:101C0000FF24C0E1D7E280E390E00C171D0748F005
:101C100031E0F32E0C1B1D0B01960C171D07D0F79E
:101C200009C0FF2039F48033910521F4C130D1057A
:101C300009F080E20E94910DCE016AE070E00E94FE
:101C4000321EEB01672BF9F6DF91CF911F910F91B7
:101C5000FF900895CF93DF93EC01FC0121968491CE
:101C6000882339F00E94910DFE01219684918823EA
:101C7000C9F7DF91CF9108958CEE91E00E942A0E72
:101C80000895CF93DF93EC018881882331F0899107
:101C90000E94910D88818823D1F7DF91CF9108951B
:101CA000A09A08958FB9779BFECF8FB19927089599
:101CB000CF9384B3836084BBC59A87B38C6287BBA0
:101CC000BC986C9A6B986D9868986998709A6E9A9F
:101CD000A998A898C3E180E00E94520EC150C7FFA6
:101CE000FACF81E38A95F1F7A89A82E08A95F1F715
:101CF000A99ACF910895A89887ED0E94520E87ED7A
:101D00000E94520E8823DCF7A89A08951F93CF9360
:101D1000DF93EC01162F0E947B0EA898112311F47B
:101D200084ED01C086ED0E94520E80E00E94520EAA
:101D30008D2F992781700E94520E8C2F0E94520E77
:101D400080E00E94520E80E00E94520EA89A9927CD
:101D5000DF91CF911F9108951F93CF93DF93EC01F3
:101D6000162F0E947B0EA898112311F483E501C061
:101D700085E50E94520ECE01880F892F881F990B8E
:101D800091958F700E94520E8C2F880F0E94520ED8
:101D900080E00E94520EA89ADF91CF911F91089582
:101DA0000F931F93CF93DF9300E010E060E0C80132
:101DB0000E94AC0EC0E0D0E060E0CE010E94860E32
:101DC0000E940506219681E0C830D807ACF30F5F6A
:101DD0001F4F88E0003018074CF3DF91CF911F911F
:101DE0000F9108951F93CF93DF93EC01162F0E945C
:101DF0007B0EA898112311F483E801C086E80E94A5
:101E0000520ECE01880F892F881F990B91958F70E4
:101E10000E94520E8C2F880F0E94520E80E00E946A
:101E2000520EA89ADF91CF911F910895CF92DF9221
:101E3000EF92FF921F93CF93DF937C01162F6A01DD
:101E4000E9010E947B0EA898112311F484E801C0D7
:101E500087E80E94520E80E00E94520E8F2D992733
:101E600081700E94520E8E2D0E94520E209739F0E2
:101E7000F60181916F010E94520E2197F7CFA89A27
:101E8000DF91CF911F91FF90EF90DF90CF90089559
:101E90000F931F93CF93DF93EC01162F042F0E9413
:101EA0007B0EA898112311F484E801C087E80E94F2
:101EB000520E80E00E94520E8D2F992781700E9451
:101EC000520E8C2F0E94520E802F0E94520EA89A02
:101ED000DF91CF911F910F910895EF92FF920F9391
:101EE0001F938C017B010E947B0EA89882E50E94C3
:101EF000520EC801880F892F881F990B91958F70FA
:101F00000E94520E202F220F8F2D99278170822B35
:101F10000E94520E8E2D0E94520E80E00E94520EA0
:101F200080E00E94520E80E00E94520E80E00E94EB
:101F3000520E80E00E94520EA89A99271F910F918D
:101F4000FF90EF900895DC01862F4115510561F057
:101F5000A40FB51F9C918927E82FFF27E151FE4F61
:101F6000849141505040B9F799270895C4988FB98A
:101F7000779BFECF6FB9779BFECFC49A0895FC0183
:101F8000C4988AE78FB9779BFECF615070408FEF7E
:101F90006F3F780729F081918FB9779BFECFF5CFFE
:101FA000C49A0895C498962F9F71982B9FB9779BD8
:101FB000FECF1FB8779BFECF67FF03C01FB8779B8C
:101FC000FECF8FB1C49A99270895FC01C4988AE383
:101FD0008FB9779BFECF615070408FEF6F3F7807CE
:101FE00031F01FB8779BFECF8FB18193F4CFC49AA5
:101FF0000895482F99278076907020910D033327FC
:102000008217930781F0407640930D0363E08FEBD6
:102010000E94B60F80910D03829586958770682F78
:102020008FE90E94B60F089508950F931F93182FFC
:10203000062F0E94F90F1F71602F812F80640E946C
:10204000B60F1F910F910895EF92FF920F931F9378
:102050007C018B0160E082E00E94151060E083E06B
:102060000E941510602F86E00E941510812F99277D
:10207000682F87E00E94151060E08AE70E94B60F83
:10208000B801C7010E94BF0F60E88FE90E94B60F38
:1020900060E88FEB0E94B60F6CE08FE90E94B60FEC
:1020A0001F910F91FF90EF9008951F93182F0E949A
:1020B000F90F612F80E00E94D20F99271F91089598
:1020C0000F931F938B01682F84ED0E941510602FD2
:1020D00086ED0E941510812F9927682F87ED0E94A9
:1020E00015108AEE0E94551080FDFBCF1F910F91B5
:1020F00008950F931F93682F84ED0E94151061E0DF
:1021000082ED0E9415108AEE0E94551080FDFBCFD3
:1021100060E082ED0E94151089ED0E94551099270C
:10212000182F002788ED0E9455109927802B912B9E
:102130001F910F910895EF92FF920F931F93CF93EA
:10214000DF937C018B018CE10E94551086FD03C05A
:1021500080E090E063C080910E0390910F03682FA0
:1021600080E00E94151080910E0390910F03892F3B
:102170009927682F81E00E94151060E08AE30E9491
:10218000D20F992790930F0380930E0360E08AE3A8
:102190000E94D20F9927382F222780910E03909109
:1021A0000F03822B932B90930F0380930E0360E019
:1021B0008AE30E94D20FC82FDD2760E08AE30E94E5
:1021C000D20F9927982F8827C82BD92B60E08AE354
:1021D0000E94D20F60E08AE30E94D20F0C171D0705
:1021E00008F4E801BE01C7010E94E50F80910E03CB
:1021F00090910F03682F8CE00E94151080910E03C0
:1022000090910F03892F9927682F8DE00E94151058
:1022100060E48EE90E94B60FCE010497DF91CF9162
:102220001F910F91FF90EF900895FF920F931F93CE
:10223000CF93DF938FEF80930D0387B3886187BBC4
:10224000C49AC79A87B3806B87BBBE9880E58DB967
:1022500081E08EB9C398E0E0F8E4CF010197F1F78F
:10226000C39A83E98A95F1F7CF010197F1F78DE1E0
:102270000E94551080FFFBCF82E096E090930F0301
:1022800080930E0390930F0380930E03C5E0D3E079
:102290008E010F5F1F4F7AE2F72EF8018491FE0145
:1022A0009491682F892F0E941510FEEFFF0E0E5F8C
:1022B0001F4F2296F7FEF1CF60E071E080E10E94AF
:1022C000601060EC8BE10E94151064E08FE90E94C1
:1022D000B60F62E774E084E10E946010DF91CF9155
:1022E0001F910F91FF900895C4988FB9779BFECFEF
:1022F0001FB8779BFECF1FB8779BFECF8FB1C49AD4
:1023000099270895E0E2F3E089E010827396815006
:1023100087FFFBCF089590E020E030E0E0E2F3E0BB
:1023200080817396882371F09F5F2F5F3F4F9A30B3
:10233000B8F390E020E030E0E0E1F3E0808988301D
:1023400019F4108AC90108959F5F73962F5F3F4F5C
:102350009A30A0F38AE090E0089508951F93CF93F8
:10236000DF9310E0C0E1D3E08889882399F0898960
:102370008150898B882371F4888B81E393E00E94DC
:102380002A0E812F0E94AD0D80E593E00E942A0E57
:102390000E943C0E1F5F63961A3030F3DF91CF919D
:1023A0001F9108956F927F928F929F92AF92BF92EA
:1023B000CF92DF92EF92FF920F931F93CF93DF9311
:1023C0004C01E62EF42E3901062F112783E190E00F
:1023D000089FE001099FD00D189FD00D1124C05F08
:1023E000DC4F2C813D814E815F8120708091000304
:1023F00090910103A0910203B0910303807028170C
:1024000039074A075B0789F082E693E00E942A0EAB
:102410006C817D818E819F810E94D20D8CE693E03C
:102420000E942A0EE6EFF2E006C083E1689FF00109
:102430001124EC5EFC4F60817181828193810E9446
:102440007B07AC018F5F9F4F39F58FE893E00E94C7
:102450002A0E83E190E0089FF001099FF00D189F7C
:10246000F00D11248F01005F1C4FF801648175810C
:10247000868197810E94D20D85EA93E00E942A0E00
:102480000E943C0EF8014481558166817781C40128
:1024900006960E94A207AC0124E130E0620E731E92
:1024A0002E2D332783E190E0289F5001299FB00C07
:1024B000389FB00C112480E193E0A80EB91ECA0128
:1024C00063E0880F991F6A95E1F7840F951F840FC9
:1024D000951F8E529D4F23E1E29EB00111246C5E48
:1024E0007C4F630146E0E42EF501008111812281D9
:1024F0003381AC01C4010E94B606F501828193814B
:10250000892F9927F40182A3F5018281F40183A325
:10251000F50180819181892F9927F40184A3F50128
:102520008081F40185A3F50140855185628573851D
:10253000C40186960E94890AF50144855585668501
:102540007785C4018A960E94890A80E5F40186A7EE
:10255000F7A682E080AB86E381AB12AA13AA14AA85
:1025600015AA26E030E0620E731EC301AA27BB271E
:10257000E2E0F0E06E0E7F1E9C01AD01B301C401EC
:102580004A960E949C0A9C01832F9927F40182ABF2
:1025900023AB2AE130E0620E731EB301C4010E9436
:1025A000100ADF91CF911F910F91FF90EF90DF9074
:1025B000CF90BF90AF909F908F907F906F90089535
:1025C0002F923F924F925F926F927F928F929F9243
:1025D000AF92BF92CF92DF92EF92FF920F931F9331
:1025E000CF93DF93CDB7DEB722970FB6F894DEBF57
:1025F0000FBECDBF4C014A960E94200A1B012C0140
:10260000F40182A19927F82EEE2483A19927E82AC4
:10261000F92A84A19927B82EAA2485A19927A82A46
:10262000B92AD7A4FFE3DF228401025E1F4FC8014D
:102630000E94200A9B01AC0180910003909101034C
:10264000A0910203B0910303281739074A075B07DB
:1026500071F081ED93E00E942A0EC8010E94200AC9
:10266000DC01CB01BC01CD010E94D20DD6C21A8281
:1026700040E1642E43E0742EF3018089882309F43D
:102680006AC2808191818E159F0509F064C28481A0
:102690009581A681B78182159305A405B50509F03A
:1026A0005AC28FEE93E00E942A0E8A810E94AD0DDD
:1026B0008DEF93E00E942A0E8CE3F301818B0D2DA8
:1026C0001127C801969587959695879521E0A22EAA
:1026D000B12CA822B92280FD95C280899927863025
:1026E000910509F4F3C18730910554F484309105C4
:1026F00029F1853091050CF0A8C1039789F019C222
:102700008830910509F408C2883091050CF407C29D
:102710008930910509F46FC10A9709F491C109C282
:10272000F0E1DF1631F484E0F301808B8AE294E07B
:10273000FDC1F301108A86E394E0F8C194012A5D9B
:102740003F4F9AE2E92EF12CE80CF91C00FF23C060
:102750008AE0F301808BC9010E945E0ADC01CB0193
:102760000196A11DB11DF30184879587A687B787C0
:10277000C7010E945E0ADC01CB01F30180879187CB
:10278000A287B387950141E16A81C4010E94D211F9
:102790008DE394E0CBC1C7010E945E0A7B018C01EE
:1027A000F30180859185A285B385E816F9060A07AD
:1027B0001B07F9F0F1E0EF16F10401051105C9F06E
:1027C00086E494E00E942A0EC7010E94FA0D80E27E
:1027D0000E94910DF301808591850E94FA0D80E29F
:1027E0000E94910D0E943C0EF301E086F186028763
:1027F0001387C40186960E945E0A7B018C01F40156
:102800008685282F33272F703070220F331F220F19
:10281000331F86A59927807F90709595879595950C
:102820008795280F391F80899927D82ECC24818934
:102830009927C82AD92AEEE0AE2EB12CA20EB31EDB
:10284000C21AD30AF30184859585A685B785E81653
:10285000F9060A071B0711F10097A105B105F1F070
:10286000E816F9060A071B0768F48E199F09A00BE2
:10287000B10BA80EB91EC81AD90A8EE694E00E94C0
:102880002A0E0CC08DE994E00E942A0E20E030E070
:1028900040E16A81C4010E94D211C1C1F9E5AF16BD
:1028A000F2E0BF0620F078E5A72E72E0B72EC50152
:1028B0008C0D9D1D8955924010F0CC24DD2496018D
:1028C00044275527F30184859585A685B785820F12
:1028D000931FA41FB51F84879587A687B78785ECAC
:1028E00094E00E942A0EC6010E94FA0D84ED94E045
:1028F0000E942A0EC114D10411F00E943C0EC501A1
:102900008C0D9D1DA816B90670F47501E80CF91C14
:102910008C010A191B09F70181917F010E94910D19
:1029200001501040C1F70E943C0E198200E010E0F7
:10293000F301828193818035910519F085509D4086
:1029400051F48E010F5F1F4F2A81A601B501C4010A
:102950000E9461168C01898199278230910589F046
:10296000833091051CF4019721F0E9C0039761F1D0
:10297000E6C020E030E040E16A81C4010E94D2114B
:10298000DEC0980140E16A81C4010E94D211980121
:1029900044275527F30180859185A285B385820F51
:1029A000931FA41FB51F80879187A287B3878BEDE4
:1029B00094E00E942A0EF301808591850E94FA0D11
:1029C0008DE50E94910DBBC085E0F301808B20E076
:1029D00030E049E16A81C4010E94D211F30180858F
:1029E0009185A285B3850196A11DB11D8087918730
:1029F000A287B387A4C08AE0F301808BC4018696C6
:102A00000E945E0ADC01CB010196A11DB11DF301FC
:102A100084879587A687B787C4018A960E945E0A35
:102A2000DC01CB01F30180879187A287B3879501F1
:102A300041E06A81C4010E94D2118EED94E076C01B
:102A4000F301108A87EE94E071C0C40186960E945B
:102A50005E0ADC01CB010196A11DB11DF301848743
:102A60009587A687B787C4018A960E945E0ADC0113
:102A7000CB01F30180879187A287B38788EF94E029
:102A80000E942A0EF1E0DF1661F487E0F301808BEB
:102A9000950140E16A81C4010E94D21184E095E071
:102AA00045C0F1E1DF1661F488E0F301808B950108
:102AB00040E16A81C4010E94D2118CE095E036C0E9
:102AC00086E0F301808B87E195E030C0C4018696F3
:102AD0000E945E0ADC01CB010196A11DB11DF3012C
:102AE00084879587A687B787C4018A960E945E0A65
:102AF000DC01CB01F30180879187A287B38700FFB8
:102B00001EC088E0808B950140E16A81C4010E946B
:102B1000D21181E295E00AC087E395E007C004FF87
:102B20000EC088E0F301808B81E595E00E942A0EBB
:102B300006C085E695E00E942A0EF301108A0E94E5
:102B40003C0EF3018089883009F069C085E0818BF3
:102B50008FE895E05BC0FA81FF5FFA8383E190E044
:102B6000680E791EFA3008F487CD92E0D91609F084
:102B700050C00E948B118A838A3008F04AC0282FE7
:102B8000332783E190E0289F8001299F100D389F13
:102B9000100D1124005F1C4F83E0F801808BE08250
:102BA000F1822482358246825782A282B382C40196
:102BB00086960E945E0ADC01CB010196A11DB11D23
:102BC000F80184879587A687B787108611861286B5
:102BD00013868CE3818B128A20E030E042E16A8127
:102BE000C4010E94D21181E090E0A0E0B0E0F801C1
:102BF00080879187A287B3878A810E9431168EEAE7
:102C000095E009C0F301108A83E094E00E942A0E47
:102C100006C08DEC95E00E942A0E0E943C0E229682
:102C20000FB6F894DEBF0FBECDBFDF91CF911F91DD
:102C30000F91FF90EF90DF90CF90BF90AF909F905B
:102C40008F907F906F905F904F903F902F9008955E
:102C5000EEECF3E089E010823596815087FFFBCFE0
:102C600008958A3058F49927FC01EE0FFF1FEE0FEC
:102C7000FF1FE80FF91FE253FC4F108208950895DB
:102C8000FC0101962491222359F0DA01A60FB71F07
:102C90002D934F5F5F4FFC01019624912223C1F7D2
:102CA000CA010895FC0106C02115310531F02150FB
:102CB0003040319684918823B9F7CF010E944016A5
:102CC00008952F923F924F925F926F927F928F92D0
:102CD0009F92AF92BF92CF92DF92EF92FF920F93AB
:102CE0001F93CF93DF93CDB7DEB72E970FB6F8942F
:102CF000DEBF0FBECDBFAA24BB2465014C011B0162
:102D00004C875D872E8728018EEA97E00E942A0E65
:102D10002E85622E772483E190E0689E7001699E83
:102D2000F00C789EF00C112480E193E0E80EF91E7F
:102D3000F7018085918501970E94FA0D8AEC97E052
:102D40000E942A0E8301000F111F000F111F060D94
:102D5000171D02531C4FF80180819927833091057C
:102D600009F4F7C1843091055CF48130910509F4D0
:102D700099C1823091050CF0E8C1892B49F003C25A
:102D8000863091050CF4ECC1069709F4F6C1FBC13D
:102D9000F401E20DF31D8081873409F0D7C08181F1
:102DA000853409F0D3C08281843509F0CFC0A101F8
:102DB0004D5F5F4F7E010894E11CF11CF70117E0A5
:102DC0001192115017FFFCCFE9E0F0E0EC0FFD1F6E
:102DD00012E01192115017FFFCCF10E0F401E40F44
:102DE000F51F8081803221F44F5F5F4F3196F9CF1C
:102DF000D401A40FB51F8C91803279F18D3069F127
:102E00008A3059F16C857D85620D731D4617570711
:102E100020F59D01F701E10FF11D80838E3239F419
:102E20008A8589878B858A878C918B8707C0183024
:102E300008F41F5F89818F3209F411504F5F5F4F93
:102E40002F5F3F4FD9018C91803239F08D3029F0BE
:102E50008A3019F046175707E8F27E010894E11C02
:102E6000F11CF701E10FF11D80818E3209F410820F
:102E700080ED97E00E942A0E10E08981882371F08E
:102E8000F701E10FF11D80810E94910D1F5F183045
:102E900028F4F701E10FF11D8081F0CF8EE20E944E
:102EA000910D10E089858823A1F0E9E0F0E0EC0FB6
:102EB000FD1FE10FF11D80810E94910D1F5F1330F6
:102EC00040F4E9E0F0E0EC0FFD1FE10FF11D80811F
:102ED000EACF88ED97E00E942A0E89818F3249F06F
:102EE000BE016F5F7F4F8DED97E00E94681B8823C6
:102EF00061F0F301EE0FFF1FEE0FFF1FE60DF71D50
:102F0000E253FC4F81E090E038C0BE016F5F7F4F1D
:102F100083EE97E00E94681B882361F0F301EE0FB7
:102F2000FF1FEE0FFF1FE60DF71DE253FC4F82E07F
:102F300090E023C0F301EE0FFF1FEE0FFF1FE60D21
:102F4000F71DE253FC4F1182128219C08081803537
:102F5000B1F481818F3499F48281833581F4838146
:102F6000843569F4F301EE0FFF1FEE0FFF1FE60D2E
:102F7000F71DE253FC4F8FEF9FEF81839283A101F6
:102F80008C859D85820D931D4817590708F0FBC05D
:102F9000AB2CBC2CCD2CF401E40FF51FD080FDE050
:102FA000AF1609F07CC02AE0B21609F078C0CF163F
:102FB00009F075C0D21609F072C046E350E08E8564
:102FC000082F1127F801EE0FFF1FEE0FFF1FE00F74
:102FD000F11FE253FC4F8181928182309105A1F073
:102FE0008330910518F4019729F035C08F5F9F4F0A
:102FF000A9F031C0B4018FE697E00E944016AC0101
:10300000B40184E297E02CC0B4018FE697E00E94FF
:103010004016AC01B4018AE197E022C083E08083CE
:10302000B4018FE697E00E944016AC01B40184E23F
:1030300097E00E944016AC01B40185E197E00E9440
:103040004016AC01B4018AEE97E00E94401622E0DF
:10305000F201208375C046E350E0B4018EE297E0B0
:103060000E944016AC01B40185E197E00E94401631
:10307000AC0182E0F2018083F80102C0EE0FFF1F75
:103080008A95E2F7E00FF11FE253FC4F81E0808365
:10309000CA018219930901968383948350C04F5FBC
:1030A0005F4F72CFF801838194810E94FA0DF7017E
:1030B000E084F184F80183819481E81AF90A82E0BE
:1030C000F2018083F801818192818130910519F0AC
:1030D000029761F01AC080E098E00E942A0E9701E2
:1030E00046E350E0B4018DE396E019C089E098E032
:1030F0000E942A0E870122E232E046E350E0B4014A
:1031000080E090E00E947E190CC084E198E00E946B
:103110002A0E970146E350E0B4018AEF95E00E9441
:103120005216AC01892B71F0F301EE0FFF1FEE0F69
:10313000FF1FE60DF71DE253FC4F82E08083CA01BA
:10314000C69726C082E292E023C0F801108283E095
:103150001BC08EE2F40186AB82E0F20180830AC0DC
:103160008EE2F40186AB82E0F2018083F70182896E
:103170008F5F828B81E090E00BC083E0F20180835F
:10318000F701128A03C081E0F201808380E090E0C1
:103190002E960FB6F894DEBF0FBECDBFDF91CF9154
:1031A0001F910F91FF90EF90DF90CF90BF90AF9065
:1031B0009F908F907F906F905F904F903F902F9057
:1031C000089508956F927F928F929F92AF92BF92CF
:1031D000CF92DF92EF92FF920F931F93CF93DF93E3
:1031E000C0E0D0E030E0632E30E0732E88249924D4
:1031F0005401CE01969587959695879502E810E043
:10320000081B190BC801AA2797FDA095BA2FBC016E
:10321000CD010E94C51C6B017C0117FF08C020E096
:1032200030E040E857E40E94181C6B017C01C501A6
:10323000B4010E94C51CD7FF06C020E030E040E882
:1032400057E40E94181C23EC35EF48E450E40E9438
:10325000121DDC01CB0120E030E040EF51E4BC0165
:10326000CD010E94621CDC01CB01BC01CD010E949A
:10327000601DDC01CB0120E030E040EA52E4BC01FB
:10328000CD010E94121DDC01CB0123EC35EF48E497
:1032900050E4BC01CD010E94621CDC01CB019C0109
:1032A000AD01C701B6010E94181CDC01CB01BC01B5
:1032B000CD010E94A81CDC01CB01682FC3010E9434
:1032C0000C1C21960894811C911CA11CB11C089413
:1032D000611C711C81E0C032D80708F48ACFDF91ED
:1032E000CF911F910F91FF90EF90DF90CF90BF9003
:1032F000AF909F908F907F906F9008952F923F9204
:103300004F925F926F927F928F929F92AF92BF92F5
:10331000CF92DF92EF92FF920F931F93CF93DF93A1
:10332000CDB7DEB728970FB6F894DEBF0FBECDBF7E
:1033300089839A836B837C834A01390128012EEAB1
:1033400039E00F8318870E331105F0F4DB01A80D67
:10335000B91D1197F9012F5F3F4F0894811C911CF3
:10336000849111968C930894411C511C0894610817
:1033700071086114710409F4EAC08F81988501967F
:103380008F839887CE9730F3F201FE97EF83F8870B
:103390002F01E834F10528F52FEFAB81BC81A80D92
:1033A000B91D74010894E11CF11CC201019683014E
:1033B000015010404F8158854330510510F41C9244
:1033C00001C02C9347012C0138010115110509F4A6
:1033D00002C18F81988501968F83988788349105E3
:1033E000E0F2E8EBFFEF4E0E5F1E28E430E0C20192
:1033F000B9010E94321E5B01629FC001639F900D64
:10340000729F900D11249201281B390B2F8338874E
:103410008CEE99E00E942A0EC5010E94FA0D80EF01
:1034200099E00E942A0E8F8198850E94FA0D65010D
:10343000CC0CDD1CCA0CDB1C49E158E0C40ED51EC7
:103440008F8198858330910510F4C80ED91E88E8C5
:1034500090E08A199B095C0192E0A916B10408F476
:1034600090C0EBE5AE16B10451F52F8138852834B4
:10347000310508F07CC0AB81BC81A80DB91D4F811E
:1034800058854330510530F4F6010894C11CD11C15
:10349000149101C01FEF1D930894811C911C089486
:1034A000610871086114710409F451C08F81988515
:1034B00001968F8398878834910508F358C0EF816F
:1034C000F885E834F10508F052C01F0153E0220CE2
:1034D000331C5A95E1F72B813C81280D391D2D8332
:1034E0003E834F8158854330510530F4F6010894EE
:1034F000C11CD11C14911DC010E007E07101110F17
:10350000C70196958795E981FA818E0F9F1F0E94CA
:10351000041C9927A816B90609F41F5F01500894E6
:10352000E11CF11C07FFEBCFFF81F0FF02C0A0FC04
:103530001160ED81FE811193ED83FE830894811C5F
:10354000911C0894610871086114710411F49301CD
:1035500050C02F8138852F5F3F4F2F83388748E039
:1035600050E0240E351E2834310508F4BACF1F82EE
:1035700018860894A108B10852E0A516B10408F015
:1035800070CFC2010E94FA0DC201805B95420E9479
:10359000FA0D1F821886AB81BC81A80DB91D74017C
:1035A0000894E11CF11C8301015010408F81988523
:1035B000039710F41C9202C08FEF8C9347018EE2A8
:1035C0000E94910D38010115110539F4EF81F8853C
:1035D000E734F10558F498010CC02F8138852F5F2E
:1035E0003F4F2F83388728343105A8F2970126539F
:1035F0003040C90128960FB6F894DEBF0FBECDBF8C
:10360000DF91CF911F910F91FF90EF90DF90CF90BE
:10361000BF90AF909F908F907F906F905F904F90F2
:103620003F902F900895CF92DF92EF92FF920F93E9
:103630001F93CF93DF93EC017B0120E030E0FB018F
:103640008081882309F439C0FE0194916901F70152
:10365000E20FF31F8081891749F521962F5F3F4FB5
:10366000FE01949121979923E1F0F701E20FF31FF6
:1036700080818917B1F48F01892F0E94910D8DE30C
:103680000E94910DF80181918F010E94910D0E947D
:103690003C0EFE019491992321F0F8018081891755
:1036A00059F3992311F4C6010AC096012F5F3F4FC9
:1036B0002196F701E20FF31FC3CF8FEF9FEFDF914A
:1036C000CF911F910F91FF90EF90DF90CF900895D1
:1036D000CF93DF939C01DB0140E08C9116C0F90190
:1036E00084918823A1F0ED01C40FD11DF9019491BB
:1036F0008881891719F080E090E00BC02F5F3F4F61
:103700004F5FFD01E40FF11D8081882341F781E0C7
:1037100090E0DF91CF910895089524E02093200355
:1037200020E530E0309311032093100324EC32E2C3
:103730004CEE50E42093140330931503409316038A
:103740005093170320E93CE93093130320931203AD
:1037500010921C0310921D0310921E0310921F035F
:10376000109218031092190310921A0310921B035F
:103770002CE32093210320E030E042E060E00E944F
:10378000D21181E090E0A0E0B0E080931803909324
:103790001903A0931A03B0931B030895EF92FF92AD
:1037A0000F931F937C0184EF99E00E942A0EC701BA
:1037B00086960E945E0ADC01CB010196A11DB11D17
:1037C00080931C0390931D03A0931E03B0931F03CB
:1037D00081E090E0A0E0B0E080931803909319039B
:1037E000A0931A03B0931B0346E350E0B70182E0B5
:1037F0009AE00E94401622E0F8012083C6971F91AC
:103800000F91FF90EF900895E199FECF9FBB8EBB83
:10381000E09A99278DB30895E199FECF9FBB8EBBA7
:103820006DBB0FB6F894E29AE19A0FBE0895505816
:10383000192ED5D001D0B8C0BA1762077307840714
:103840009507B1F188F40EF410940B2EBA2FA02D29
:10385000062E622F202D072E732F302D082E842F39
:10386000402D092E952F502DFF275523B9F0591BB8
:1038700049F0573E98F0469537952795A795F04023
:103880005395C9F776F0BA0F621F731F841F30F487
:10389000879577956795B795F040939517FA0F2E12
:1038A0000895BF1BBB27BA0B620B730B840BF6CFBB
:1038B000DEF6B2C0592F482F372F262F9FE380E81E
:1038C000772766278CD001D06FC0552359F09923F4
:1038D00069F09F575F57951B33F442F4903811F409
:1038E000915805C079C091589F3F09F495C0BB27F6
:1038F000112462177307840730F4660F771F881F3F
:10390000BB1F915098F311D00F920FD00F920DD092
:10391000A0E82617370748071B0609F0A048BA2F6A
:10392000602D7F918F9100240895A0E800246217F4
:1039300073078407B10528F0621B730B840BB10970
:103940000A2A660F771F881FBB1FA69581F7089567
:1039500097FB51D09F3738F0FEE9F91B982F872F3E
:10396000762F6B2F05C055C09695879577956795EF
:10397000F150D0F73EF490958095709561957F4F0A
:103980008F4F9F4F0895E89403C097FB0EF4F3DF29
:10399000B62F672F782F892F9EE9002405C09A95AE
:1039A000BB0F661F771F881F11249923A1F088235E
:1039B000B2F79F3F59F0BB0F48F421F4002011F4F7
:1039C00060FF04C06F5F7F4F8F4F9F4F881F979599
:1039D000879597F908951DC09FEF80EC0895052EF7
:1039E000092607FA440F551F5F3F79F0AA27A5174C
:1039F00008F051E04795880F991F9F3F31F0BB2792
:103A0000B91708F091E0879508959F919F9111242F
:103A1000E3CF66277727882799270895592F482FBE
:103A2000372F262FDCDF01D0BFCF992339F0552364
:103A300029F09F575F57950F13F4CAF1EDCF9158B6
:103A40009F3FE1F3A62F00241124BB2766275527AB
:103A5000F8E0A69520F4020E131EB41F651F220F76
:103A6000331F441F551FFA95A1F7F8E0E72F77277A
:103A7000F8E0E69520F4130EB41F651F7A1F330F8C
:103A8000441F551FAA1FFA95A1F7F82F8827F6950E
:103A900020F4B40F651F7A1F8E1F440F551FAA1FF5
:103AA000EE1FFF23A1F788231AF4939539F494CFDE
:103AB000000C111CBB1F661F771F881F012808956B
:103AC0009F939F77993358F050E449EC3FE02BEDFA
:103AD0000AD05FEB49EC3FE02BEDAADE17D05F91F7
:103AE0005078952708955F77552319F444230AF0F9
:103AF00073CF2F933F934F935F93E4DE5527442773
:103B00006FD05F914F913F912F918CCF1F939F77F3
:103B100050EC49E43FE02BED8BDE10E89F775FE34C
:103B200049EC3FE02BED621773078407950720F0FF
:103B300050EC49E47DDE112771DF9068E4E5F0E0A8
:103B400003D091271F910895092E55DFFF92EF9220
:103B5000DF92CF92BF92AF92B02CC92ED82EE72E13
:103B6000F62EA59018D0A590AA2071F09F938F9360
:103B70007F936F936F2D7E2D8D2D9C2D0CD02F91CB
:103B80003F914F915F91A1DEAF90BF90CF90DF90BA
:103B9000EF90FF9009CF55D047FB406804C02F2D10
:103BA0003E2D4D2D5C2DEF93FF933FDFFF91EF9165
:103BB00048D0AA2707F80B24102C042607FA4068DF
:103BC000FF933ADEFF91992341F0882332F09A95D2
:103BD000BB0F661F771F881FF8CFAA9401F70895BF
:103BE00097FB09DFCF93DF93D52FC42F55274427A9
:103BF000332722279923D9F09F37C8F0F92FD4DE35
:103C0000592F482F372F262FF63968F4A1DEBDDE55
:103C1000C030CD0721F06993799389939993905897
:103C2000DF91CF9105CE9927882777276627C03067
:103C3000CD0721F02993399349935993DF91CF917F
:103C4000B3CE55914591359125910895991B79E011
:103C500004C0991F961708F0961B881F7A95C9F71C
:103C600080950895AA1BBB1B51E107C0AA1FBB1F6B
:103C7000A617B70710F0A61BB70B881F991F5A95F8
:103C8000A9F780959095BC01CD010895A1E21A2E67
:103C9000AA1BBB1BFD010DC0AA1FBB1FEE1FFF1FF0
:103CA000A217B307E407F50720F0A21BB30BE40B40
:103CB000F50B661F771F881F991F1A9469F7609587
:103CC0007095809590959B01AC01BD01CF01089541
:103CD0003F3F3F203A2069702070726F746F200060
:103F00000895F894C09A5FD04427E0E0F0E080E2A2
:103F1000242F3DD055272BD0202F539528D0302F3C
:103F2000539507D05523B9F743950EE1041780F751
:103F3000FFCF022E132E21E011D032968A9569F41C
:103F4000E054F04023E00AD025E008D021E106D07B
:103F500020E4E20F08F4F39580E2089507B700FD2E
:103F6000FDCFF894E199FECF27BFE89508951ED0C4
:103F7000A89804ED23D0002721D000271FD0052FBB
:103F80001DD000271BD0002719D0A89A08950ED065
:103F9000A89803E513D0002727FD01600FD0022F5A
:103FA000000F0CD000270AD0A89A0895A89807ED12
:103FB00005D004D007FFFDCFA89A08950FB9779BCD
:103FC000FECF0FB1089505E008BB03E004BBA9983C
:103FD000A89A0CE207BB01E50EB9A89AA99A089520
:00000001FF
